:020000040000FA
:040000009DEF00F080
:02000800AFD077
:08001800FDD00E6E960E066E7F
:10002000980E076E55D8D8B4CA90D8A4CA80FC0FD1
:10003000D8A0CA92D8B0CA82800E066E960E076EFD
:10004000980E0A6E0B6ACAB025D8CAB223D842D815
:100050000604CB6E06C008F007C009F000500C6E15
:100060000D6E003C0D6A4BD80B500E2E0AD0BE6EA2
:100070000C0EBD6E0ABEBD8A0ABCBD889394CA84AC
:100080001200BB6E0C0EBA6E0ABEBA8A0ABCBA88DF
:100090009492F5D700D8D8900A320732063212006F
:1000A000096A086EFF0E0826092200D0D8A01200A7
:1000B000030E076EE70E02D8F5D7076AFE0F066E2D
:1000C000E86A075AD8A012000000060600D0F8D748
:1000D0000B6A0A6A100EF36E07340A360B360850A4
:1000E0000A5C09500B5805E308500A5E09500B5A88
:1000F000D88006360736F32EEFD706501200085088
:100100000C02F3CF0AF0F4CF0BF009500C02F350BD
:100110000B2608500D02F3500B260A501200086AF5
:10012000096A04D00732063208360936FF0FFAE2B0
:1001300009C007F00850066E1200F86A4F0EAF6E45
:10014000240EAC6E900EAB6E0001070EB46E0F0E57
:10015000C16EC69AC10E926EE00E936EC00E946E82
:10016000956AE80E966EA5D09EAA1BD0060EAB141B
:1001700012E1E1CF47F0E2CF48F0492A1EEE80F0CD
:100180004950E126000EE222AECFE7FF47C0E1FF73
:1001900048C0E2FF1100AE50AE50AB98AB881100E2
:1001A0000AD0F2A408D0F294114A122A817A106A75
:1001B000D6CF0FF01100110049504A5C14E04A2AD2
:1001C000E9CF06F0EACF07F00EEE80F04A50E926BC
:1001D000000EEA22EF50066E06C0E9FF07C0EAFFF4
:1001E000D880120004D0E868066ED8A01200120071
:1001F000496A4A6A9D8A9F8AF28EF28C12009D9A01
:100200000EEE80F0000EEE6AE82EFDD7496A4A6ACB
:100210009D8A1200F29ED8CF5AFEE8CF5BFEE0CF57
:100220005CFEE9CF5DFEEACF5EFEE1CF5FFEE2CF8E
:1002300060FED9CF61FEDACF62FEF6CF63FEF7CF64
:1002400064FEF5CF65FEF3CF66FEF4CF67FEA6CF62
:1002500068FEF28E0001A19236A204D0154A162A39
:1002600015A200D0156A166AF29E5ACED8FF5BCE50
:10027000E8FF5CCEE0FF5DCEE9FF5ECEEAFF5FCE39
:10028000E1FF60CEE2FF61CED9FF62CEDAFF63CE3E
:10029000F6FF64CEF7FF65CEF5FF66CEF3FF67CEBF
:1002A000F4FF68CEA6FFF28E10009EA8FED7AD6EBA
:1002B0001200939A8A8A0A0EF3DE939A8A9A93948A
:1002C0008A8493968A869292899292948994366AC5
:1002D00096948D9496928D9296908D9000688A0E49
:1002E000086E090E096E010E98DE00688A0E086E0F
:1002F000090E096E020E91DE3968F3EC05F08FEC01
:1003000005F0B8EC06F0F8EC06F0949A8B8A949815
:100310008B984590406A030E3F6EF80E3E6E3D6A24
:10032000416A040E426E94908B8062DF68DFCD6A72
:10033000F294F28A870ED56EB16AA192A082B26A57
:10034000B36AD08EA292B10EB16E3C0EC26E0E0E8A
:10035000C16E820EC06EC280A1EC05F08B902CDFC6
:10036000176EEB0E175C05E3FE0E175C01E21B6ACD
:1003700003D217AE21D01B6A8A0E175C05E117C0A5
:100380001BF01C681D6817D09A0E175C05E117C09A
:100390001BF01E6824680FD0BA0E175C05E117C069
:1003A0001BF02568266807D0EA0E175C04E117C029
:1003B0001BF027682868E0D11B5202E1DDD1DCD1B7
:1003C0008A0E1B5C36E11C2803E117C01CF02FD0FD
:1003D00017C01DF0270E1C5C29E3580E1C5C26E29A
:1003E0008D908B9040BE16D03D503E103F10401077
:1003F00011E0D6CF0FF0D7CF10F03D500F242A6E6A
:100400003E5010202B6E3F5011202C6E4050122079
:100410002D6E368036A206D045B0828845A08298DF
:1004200036928992369489948B9A8B861C68A4D1D3
:10043000A3D19A0E1B5CD8A47CD11E2803E117C05F
:100440001EF076D117C024F024522DE1270E1E5C39
:1004500029E3580E1E5C26E28D908B9040BE16D08C
:100460003D503E103F10401011E0D6CF0FF0D7CFD7
:1004700010F03D500F242A6E3E5010202B6E3F503E
:1004800011202C6E405012202D6E368036A204D0E2
:1004900045B0828845A08298899236923694899494
:1004A0008B9A8B8645D1270E1E5CD8A040D1580E62
:1004B0001E5CD8B03CD18B801F28016E026A0236C8
:1004C0000252D8A444D001501E5CD8A440D0270EBC
:1004D0001E5C3C6E00EE4BF0D8903C34EBCF37F016
:1004E000E82AEBCF38F08A908A9237C006F0076A84
:1004F000080E15DE836E8A948A8438C006F0076A77
:10050000080E0DDE836E8A948A848A8237C006F0D4
:10051000076A080E04DE836E8A948A8438C006F067
:10052000076A080EFCDD836E8A948A848D848B9A18
:100530001EC01FF036A204D045B0828845A0829824
:10054000369236908D801EC046F08B96F0D01E50AD
:100550001F5CD8B07AD04B0E1E5CD8B045D0270EA9
:100560001E5C3C6E00EE4BF0D8903C34EBCF37F085
:10057000E82AEBCF38F08A908A9237C006F0076AF3
:10058000080E8FEC00F0836E8A948A8438C006F0DF
:10059000076A080E8FEC00F0836E8A948A848A8240
:1005A00037C006F0076A080E8FEC00F0836E8A945D
:1005B0008A8438C006F0076A080E8FEC00F0836E5C
:1005C0008A948A848D848B9A1EC01FF036A206D02E
:1005D00045B0828845A082988992369236908D8067
:1005E0001EC046F08B9630D0270E1F5C07E3270E07
:1005F0001F5C01EE0FF0EB50446E03D001010F5170
:10060000446E00011EC021F01FC020F08D908B961B
:100610008D8436A204D045B0828845A08298369257
:1006200036908B9AD6CF0FF0D7CF10F043500F24CF
:10063000326E44501020336E000E1120346E000EC6
:100640001220356E3684898472D01F501E5C3DE2C4
:1006500082788D9036908B96369489941EC023F0C4
:100660001F04226E270E225C3C6E00EE4BF0D890E9
:100670003C34EBCF37F0E82AEBCF38F08A908A92FF
:1006800037C006F0076A080E8FEC00F0836E8A947C
:100690008A8438C006F0076A080E8FEC00F0836E7B
:1006A0008A948A84D6CF0FF0D7CF10F041500F2410
:1006B0002E6E425010202F6E000E1120306E000E54
:1006C0001220316E3682898232D01E501F5C2FE19B
:1006D0008B9A8D841E50465C21E0270E1E5C3C6E7A
:1006E00000EE4BF0D8903C34EBCF37F0E82AEBCF5C
:1006F00038F08A8237C006F0076A080E8FEC00F0E7
:10070000836E8A948A8438C006F0076A080E8FECDC
:1007100000F0836E8A948A841EC046F08D8036A2D3
:1007200004D045B0828845A08298366A8B961E68B0
:1007300023D0BA0E1B5C09E1252803E117C025F080
:1007400003D017C026F093D917D0EA0E1B5C14E132
:10075000272803E117C027F00FD017C028F0400E5C
:10076000285C05E3400E285C296EFDD804D0285093
:100770004008296E3AD9276836A015D0D6CF0FF099
:10078000D7CF10F02A500F5C2B5010582C50115816
:100790002D50125812502D18D8B0800A04E78B96AD
:1007A0008B8A36901F6A36A26BD02250235C28E1D8
:1007B00023C01FF036928278270E235C3C6E00EE39
:1007C0004BF0D8903C34EBCF37F0E82AEBCF38F041
:1007D0008A8237C006F0076A080E8FEC00F0836E3D
:1007E0008A948A8438C006F0076A080E8FEC00F0FD
:1007F000836E8A948A848D8023C046F0899240D08B
:10080000D6CF0FF0D7CF10F02E500F5C2F501058CE
:10081000305011583150125812503118D8B0800A47
:100820002FE72206270E225C3C6E00EE4BF0D8909C
:100830003C34EBCF37F0E82AEBCF38F08A908A923D
:1008400037C006F0076A080E8FEC00F0836E8A94BA
:100850008A8438C006F0076A080E8FEC00F0836EB9
:100860008A948A8422C01FF041500F242E6E425079
:1008700010202F6E000E1120306E000E1220316EEF
:1008800036A46FD02050215C27E121C01FF03694A0
:10089000270E215C3C6E00EE4BF0D8903C34EBCF41
:1008A00037F0E82AEBCF38F08A8237C006F0076AC3
:1008B000080E8FEC00F0836E8A948A8438C006F0AC
:1008C000076A080E8FEC00F0836E8A948A848D800C
:1008D00021C046F0899445D0D6CF0FF0D7CF10F085
:1008E00032500F5C33501058345011583550125854
:1008F00012503518D8B0800A34E7202A270E205C21
:100900003C6E00EE4BF0D8903C34EBCF37F0E82A49
:10091000EBCF38F08A908A9237C006F0076A080E4B
:100920008FEC00F0836E8A948A8438C006F0076AE0
:10093000080E8FEC00F0836E8A948A8420C01FF02A
:1009400001EE0FF03C50EB50446E43500F24326EDA
:1009500044501020336E000E1120346E000E122011
:10096000356EAFEF01F0E86A36B2010F36B4010F11
:10097000016E026A0250011037E100EEADF0D8902E
:100980003C34EBCF01F0E82AEBCF02F02950010212
:10099000F3CF19F0F4CF1AF00202F3501A2600EE4A
:1009A0004BF0D8903C34EBCF01F0E82AEBCF02F0CB
:1009B0001950015C376E1A500258386E37C006F075
:1009C000076A080E8FEC00F0836E8A908A928A94F0
:1009D0008A8438C006F0076A080E8FEC00F0836E38
:1009E0008A948A8436908B961200E86A36B2010F98
:1009F00036B4010F016E026A0250011037E100EEB9
:100A0000ADF0D8903C34EBCF01F0E82AEBCF02F008
:100A100029500102F3CF19F0F4CF1AF00202F3507B
:100A20001A2600EE4BF0D8903C34EBCF01F0E82AC8
:100A3000EBCF02F019500124376E1A500220386EA5
:100A400037C006F0076A080E8FEC00F0836E8A90BC
:100A50008A928A948A8438C006F0076A080E8FEC5E
:100A600000F0836E8A948A8436908B9612003D0E35
:100A7000255C1AE126520AE1396A006A8A0E086E7C
:100A8000090E096E020E0DEC00F00DD0D890263440
:100A9000396E392A39C000F08A0E086E090E096EC7
:100AA000020E0DEC00F02BD03F0E255C0AE126C0B3
:100AB0003AF03AAC03D08B88458002D08B984590B1
:100AC0001ED0410E255C0CE1406A3F6A26C03EF014
:100AD0003D6A030ED8903E363F36E82EFBD70FD046
:100AE000420E255C08E1265203E13B9018D802D063
:100AF0003B8007D804D07B0E255CD8B410D825687D
:100B000012001FD836A204D045B0828845A0829832
:100B10008D848B9A270E1F6E366A8B96120036A232
:100B200004D045B0828845A08298366A116A126A5C
:100B30008D948D901F6A206A216A8B968B908B8A88
:100B400012008B8A4BC037F04CC038F08A848A8000
:100B50008A826C0E836E8A948A848A908A9237C0C5
:100B600006F0076A080E8FEC00F0836E8A948A8480
:100B700038C006F0076A080E8FEC00F0836E8A9486
:100B80008A848A808A826E0E836E8A948A848A928C
:100B900037C006F0076A080E8FEC00F0836E8A9467
:100BA0008A8438C006F0076A080E8FEC00F0836E66
:100BB0008A948A848A826D0E836E8A948A848A904B
:100BC00037C006F0076A080E8FEC00F0836E8A9437
:100BD0008A8438C006F0076A080E8FEC00F0836E36
:100BE0008A948A8412001A0E4B6EFB0E4C6E030E12
:100BF0004D6EED0E4E6EB50E4F6EDF0E506E270E23
:100C0000516ED30E526E4D0E536EC70E546E1D0EA6
:100C1000556EBC0E566E8F0E576EB10E586E970EF7
:100C2000596EA70E5A6E2F0E5B6E9E0E5C6E4F0EA7
:100C30005D6E950E5E6EED0E5F6E8C0E606E040E38
:100C4000616E850E626E8D0E636E7D0E646E810E1A
:100C5000656E760E666EDB0E676E6F0E686E930EB7
:100C6000696E690E6A6EA60E6B6E630E6C6E0F0E69
:100C70006D6E5E0E6E6EC70E6F6E580E706ECC0E81
:100C8000716E530E726E180E736E4F0E746EA70E49
:100C9000756E4A0E766E770E776E460E786E820E01
:100CA000796E420E7A6EC70E7B6E3E0E7C6E410EE2
:100CB0007D6E3B0E7E6EED0E7F6E370E806FCA0E20
:100CC000816F340E826FD30E836F310E846F070EE7
:100CD000856F2F0E866F640E876F2C0E886FE60E61
:100CE000896F290E8A6F8C0E8B6F270E8C6F540EB6
:100CF0008D6F250E8E6F3B0E8F6F230E906F410E02
:100D0000916F210E926F630E936F1F0E946FA00E62
:100D1000956F1D0E966FF70E976F1B0E986F650EF1
:100D2000996F1A0E9A6FEA0E9B6F180E9C6F840EC5
:100D30009D6F170E9E6F320E9F6F160EA06FF30EF3
:100D4000A16F140EA26FC60EA36F130EA46FAA0E8E
:100D5000A56F120EA66F9E0EA76F110EA86FA10EA3
:100D6000A96F100EAA6FB20EAB6F0F0EAC6F120010
:100D7000186A300E185C2FE200EE4BF0D890183451
:100D8000EBCF01F0E82AEBCF02F01828056E00EE59
:100D90004BF0D8900534EBCF03F0E82AEBCF04F00A
:100DA0000350015C376E04500258386E37C001F0B2
:100DB00038C002F0070ED89002320132E82EFBD77D
:100DC00000EEADF0D890183401C0EBFFE82A02C065
:100DD000EBFF182ACEE10BC101F00CC102F001C0FB
:100DE0000DF102C00EF14BC037F04CC038F01200CC
:100DF000010E01010F6F106F116F126F136F146FDF
:100E0000156F166F176F186F196F1A6F1B6F1C6FA6
:100E10001D6F1E6F1F6F206F216F226F236F246F56
:100E2000256F266F276F020E286F030E296F040EA1
:100E30002A6F050E2B6F060E2C6F070E2D6F080EF6
:100E40002E6F090E2F6F0A0E306F0B0E316F0C0EC6
:100E5000326F0E0E336F100E346F140E356F180E86
:100E6000366F1E0E376F240E386F2C0E396F360E0C
:100E70003A6F420E3B6F4E0E3C6F5E0E3D6F700E32
:0C0E80003E6F880E3F6F00011200FFD78C
:020000040030CA
:0300010006160ED2
:020005008580F4
:060008000FC00FE00F40E5
:00000001FF
